:020000021000EC
:10F000000C9490F80C94B7F80C94B7F80C94B7F8EB
:10F010000C94B7F80C94B7F80C94B7F80C94B7F8B4
:10F020000C94B7F80C94B7F80C94B7F80C94B7F8A4
:10F030000C94B7F80C94B7F80C94B7F80C94B7F894
:10F040000C94B7F80C94B7F80C94B7F80C94B7F884
:10F050000C94B7F80C94B7F80C94B7F80C94B7F874
:10F060000C94B7F80C94B7F80C94B7F80C94B7F864
:10F070000C94B7F80C94B7F80C94B7F80C94B7F854
:10F080000C94B7F80C94B7F80C94B7F80C94B7F844
:10F090000C94B7F80C94B7F80C94B7F80C94B7F834
:10F0A0000C94B7F80C94B7F80C94B7F80C94B7F824
:10F0B0000C94B7F80C94B7F80C94B7F80C94B7F814
:10F0C0000C94B7F80C94B7F80C94B7F80C94B7F804
:10F0D0000C94B7F80C94B7F80C94B7F80C94B7F8F4
:10F0E0000C94B7F80C94B7F80C94B7F80C94B7F8E4
:10F0F0000C94B7F80C94B7F80C94B7F80C94B7F8D4
:10F100000C94B7F80C94B7F80C94B7F80C94B7F8C3
:10F110000C94B7F80C94B7F80C94B7F80C94B7F8B3
:10F1200011241FBECFEFD1E4DEBFCDBF12E0A0E0BF
:10F13000B2E0E0E9F8EF01E00BBF02C007900D92EA
:10F14000A430B107D9F722E0A4E0B2E001C01D92DB
:10F15000A630B207E1F70E94D4F80C9446FC01E413
:10F160000EBF0FEF0DBF11241FBE0C94D4F80C94EA
:10F1700000F88093C6008091C00086FFFCCF80918C
:10F18000C00080648093C000089520E030E028171C
:10F19000390749F0EFECF7E03197F1F700C00000D4
:10F1A0002F5F3F4FF4CF0895CF93DF93CDB7DEB7F6
:10F1B000C552D1400FB6F894DEBF0FBECDBF80E878
:10F1C000809361001092610001E40EBF0FEF0DBF4C
:10F1D00084B7F894A89514BE8091600088618093EC
:10F1E00060001092600078946B9A739A2298109243
:10F1F000C0001092C1008091C6008091C000826062
:10F200008093C00093E39093C40088E18093C10091
:10F210008091C00082608093C0009093C400000081
:10F220008CB1C12CD12C760167EC862E6BE1962E29
:10F23000A12CB12C78E0772E00E010E08091C00086
:10F2400087FF06C00F5F1F4F01151105A9F326C0E8
:10F2500001151105B9F725E02A95F1F700004FEFE8
:10F26000C41AD40AE40AF40A91E080E0A1E3CA16C1
:10F27000A5E7DA06E104F10408F490E0092F182F5D
:10F28000C701B601A50194010E9416FC672B682BEB
:10F29000692BA1F68EB187258EB9D0CF013011052B
:10F2A00009F0A2C2C25EDE4F1882CE51D140312C8D
:10F2B000CC5DDE4F19821882C452D140C12CD12CB2
:10F2C0007601412C512C320120E030E060E0013029
:10F2D0001105F9F080E090E0DC014091C00047FDAD
:10F2E00018C00196A11DB11D8130E2E19E07EAE739
:10F2F000AE07B10590F3812C912C5401ABBEF40103
:10F30000479156914F3F5F4F29F3EE27FF2709940E
:10F31000E1CF4091C600633009F120F4613079F00B
:10F3200040F015C0653051F1E8F0663009F446C090
:10F3300090C04B3109F46CC200E010E0C8CF342615
:10F34000C25EDE4F4883CE51D14062E0F5CF242F1C
:10F3500030E0322F2227342663E0EECF242B3426F0
:10F3600064E0EACF4E3009F05FC23426CC5DDE4F58
:10F3700019821882C452D14065E0DECFCC5DDE4FE9
:10F3800088819981C452D1400196E1E0F0E0EC0F10
:10F39000FD1FCC5DDE4F88809980C452D140E80DBE
:10F3A000F91D408334268217930709F435C2CC5DDA
:10F3B000DE4F99838883C452D140BECF431134C2FB
:10F3C0002981233109F4E2C060F5263009F4CBC06D
:10F3D00000F5223009F441C0233009F46BC021301C
:10F3E00009F0AFC11A8288E08B8381E48C8386E5C3
:10F3F0008D8382E58E8389E48F8383E5888780E52A
:10F4000089878FE58A8782E38B87212C0BE010E0C8
:10F410009DC1213109F45BC008F09DC02031E9F0A5
:10F4200090C1283109F46FC048F4253109F4AEC009
:10F4300008F432C1263109F42FC183C12A3109F4FD
:10F4400055C008F476C02B3109F445C02D3139F090
:10F4500078C1673009F4B4CF6FCF212C3AC08D81C9
:10F46000803339F49F819923B1F09130B1F497EA58
:10F4700017C0982F907599F0803521F499E0E0E05D
:10F48000F0E005C0883559F4E3E0F0E099E09093AE
:10F490005700949105C09EE103C091E001C090E047
:10F4A0001A821B828C831D829E831F82212C07E07F
:10F4B00010E04CC1EA81E059E33028F4F0E0E0507C
:10F4C000FE4F808101C080E01A828B8340C02224DD
:10F4D00023941A8239C18D81882321F0813021F44F
:10F4E00087EA24C08EE122C081E020C01A82E1E0D8
:10F4F000F0E089E080935700E491EB831C82212C9B
:10F5000004E010E023C18B81803551F48C81883078
:10F5100019F4E2E0F0E006C089E0E0E0F0E003C0CA
:10F52000E3E0F0E089E08093570084911A828B83B6
:10F53000E5CF8D81836C99E0E1E0F0E0082E9093B7
:10F540005700E89507B600FCFDCF1A821B82212CDC
:10F5500003E010E0FBC01A82212C02E010E0C12C75
:10F56000D12C7601F3C08A814B80512C612C712CF7
:10F57000320155244424782A8D81482A8C81582AC6
:10F58000440C551C661C771C1A82DDC02A80312C65
:10F59000322C22248B81282A233109F047C0C11440
:10F5A000F0ECDF06F1E0EF06F10478F483E0882E5A
:10F5B000F601E0925B0080925700E89507B600FCE8
:10F5C000FDCF2FEFD21AE20AF20A2B85B301A20176
:10F5D000CE010B9611E0DC011296CD01FD013197B1
:10F5E000E08130E03E2B0901FA0160935B0010934B
:10F5F0005700E89511244E5F5F4F6F4F7F4FE2E059
:10F600002E1A31082114310411F02C91E4CF85E039
:10F61000F20160925B0080935700E89507B600FC0A
:10F62000FDCF81E180935700E89532C0530142013C
:10F63000B694A79497948794C15EDE4F888299828E
:10F64000AA82BB82CF51D1408E01055F1F4FA12CF2
:10F65000B12CA214B30489F0D8016D918D01C15E63
:10F66000DE4F88819981CF51D1408A0D9B1D0E9428
:10F6700038FCBFEFAB1ABB0AECCFA50160E070E02D
:10F68000440F551F661F771F440D551D661D771DBE
:10F690001A822A013B0157C08A8190E0982F88275F
:10F6A0003B81832B8C010D5F1F4F1A822431A1F403
:10F6B000DE0113966BBEF201279136912C931296C0
:10F6C000FD0131973083E2E04E0E511C611C711C2C
:10F6D0000297009779F732C0FE0133969C01B3017F
:10F6E000A20141BD852E962EA72EBB24C15EDE4F02
:10F6F00088829982AA82BB82CF51D14082BC4F5F5F
:10F700005F4F6F4F7F4FF89AA0B5A19321503109F9
:10F710002115310531F7AC014150510960E070E02D
:10F720004F5F5F4F6F4F7F4F440E551E661E771E13
:10F73000A3E0B0E0AC0FBD1FA80FB91F1C92212C95
:10F7400005C080EC8A83212C02E010E08BE10E944E
:10F75000B9F8C25EDE4F8881CE51D1400E94B9F81F
:10F76000812F0E94B9F8802F0E94B9F88EE00E9484
:10F77000B9F895E1392EC25EDE4F9880CE51D14066
:10F78000392430263126CE0101965C01080F191F5D
:10F79000A016B10691F0F50191915F01892FCD5D21
:10F7A000DE4F9883C352D1400E94B9F8CD5DDE4F41
:10F7B0009881C352D1403926EBCF832D0E94B9F8EE
:10F7C000C25EDE4F2881CE51D1402F5FC25EDE4F38
:10F7D0002883CE51D1408EB198E089278EB921106F
:10F7E00003C000E010E070CD6B98739884E690E061
:10F7F0000E94C5F800008091C0008D7F8093C000FA
:10F8000081E180935700E895EE27FF270994FFCF09
:10F810008BE1382E61E090CDCC5DDE4F39832883BB
:10F82000C452D14066E088CD60E086CDA1E21A2EB8
:10F83000AA1BBB1BFD010DC0AA1FBB1FEE1FFF1F94
:10F84000A217B307E407F50720F0A21BB30BE40BE4
:10F85000F50B661F771F881F991F1A9469F760952B
:10F860007095809590959B01AC01BD01CF010895E5
:10F87000262FF999FECF1FBA92BD81BD20BD0FB6CC
:10F88000F894FA9AF99A0FBE01960895F894FFCF6A
:04F890000F020A0059
:040000031000F000F9
:00000001FF
